:100000000C942A000C9445000C9445000C94450077
:100010000C9445000C9485010C94B2010C94DA0107
:100020000C9445000C9431010C9445000C9445004F
:100030000C9445000C9445000C94FC020C94450073
:100040000C9445000C9445000C9445000C9445001C
:100050000C94450011241FBECFE5D4E0DEBFCDBF18
:1000600010E0A0E6B0E0E4EDF8E002C005900D92EB
:10007000AC36B107D9F710E0ACE6B0E001C01D9294
:10008000A03CB107E1F70C94A5000C940000CF93BD
:10009000DF93CDB7DEB7E7E3F0E08FE18083E1E304
:1000A000F0E084E08083DF91CF910895CF93DF93D8
:1000B000CDB7DEB721970FB6F894DEBF0FBECDBF28
:1000C000F89480E29EE49093BD008093BC00198276
:1000D0002FC08981482F552789819927880F991F1B
:1000E000FC01EC57FF4F808191819C0128513C4FCE
:1000F000CA01880F991FFC01E455FF4F318320830B
:100100002091BC003091BD0089819927880F991FEB
:10011000FC01E455FF4F80819181A901481B590BD7
:10012000CA019093BD008093BC0089818F5F898351
:100130008981883070F2789421960FB6F894DEBFEA
:100140000FBECDBFDF91CF910895CF93DF93CDB791
:10015000DEB721970FB6F894DEBF0FBECDBF0E9469
:1001600047000E940F010E94EE020E943D03109280
:10017000AB0089E992E090937F0080937E0087EE48
:1001800092E09093810080938000789400C08091E9
:100190007200813041F4109272008091AB0088238C
:1001A00011F40E94560080917000813081F7109206
:1001B000700019821CC080E690E00E94770389815C
:1001C00099270E94C10387E690E00E947703898106
:1001D0009927880F991FFC01E455FF4F8081918179
:1001E0000E94C1030E94B20389818F5F8983898144
:1001F000893008F3CCCFCF93DF93CDB7DEB7F89437
:10020000E9E5F0E089E180837894DF91CF9108956A
:10021000CF93DF93CDB7DEB7DF91CF910895CF9322
:10022000DF93CDB7DEB7E3E5F0E082E08083EFE473
:10023000F0E01082EEE4F0E082E08083EAE4F0E0B7
:1002400084EF91E091838083E8E4F0E080ED97E033
:1002500091838083E9E5F0E089E18083DF91CF91AC
:1002600008951F920F920FB60F9211248F93CF9380
:10027000DF93CDB7DEB78091AA008F5F8093AA008D
:100280008091AA008834C9F581E0809371001092B2
:10029000AA00809175008F5F809375008091750032
:1002A000853029F41092750081E08093720080916E
:1002B00073008F5F8093730080917300843641F4E4
:1002C0001092730081E080936E0081E08093700053
:1002D00080917300823319F481E0809370008091E3
:1002E00074008F5F80937400809174008A3029F4C9
:1002F0001092740081E080936F00DF91CF918F9115
:100300000F900FBE0F901F9018951F920F920FB66F
:100310000F9211242F933F934F935F936F937F938B
:100320008F939F93AF93BF93EF93FF93CF93DF93FD
:10033000CDB7DEB7E0917E00F0917F000995DF91A7
:10034000CF91FF91EF91BF91AF919F918F917F914D
:100350006F915F914F913F912F910F900FBE0F9032
:100360001F9018951F920F920FB60F9211248F9322
:10037000AF93BF93EF93FF93CF93DF93CDB7DEB7E8
:10038000A2E3B0E0E2E3F0E080818B7F8C93A8E30E
:10039000B0E0E8E3F0E080818F7E8C93DF91CF9135
:1003A000FF91EF91BF91AF918F910F900FBE0F9082
:1003B0001F9018951F920F920FB60F9211242F9332
:1003C0003F938F939F93AF93BF93EF93FF93CF93FD
:1003D000DF93CDB7DEB72297DEBFCDBFA2E3B0E09B
:1003E000E2E3F0E0808184608C93ECE4F0E0118241
:1003F0001082A8E4B0E080916C009927880F991FC3
:10040000FC01E455FF4F8081918111969C938E935E
:1004100080916C00882339F4A8E3B0E0E8E3F0E0D1
:10042000808180618C9380916C00282F33273A83E0
:10043000298389819A8182309105C1F129813A818C
:100440002330310554F489819A81009789F02981FC
:100450003A8121303105D9F04EC089819A818330AB
:10046000910599F129813A8124303105E9F143C0A0
:10047000A8E3B0E0E8E3F0E0808180618C93A8E33A
:10048000B0E0E8E3F0E0808181608C9334C0A8E3C1
:10049000B0E0E8E3F0E080818E7F8C93A8E3B0E0E9
:1004A000E8E3F0E0808182608C9325C0A8E3B0E0AF
:1004B000E8E3F0E080818D7F8C93A8E3B0E0E8E38F
:1004C000F0E0808184608C9316C0A8E3B0E0E8E39C
:1004D000F0E080818B7F8C93A8E3B0E0E8E3F0E06C
:1004E000808188608C9307C0A8E3B0E0E8E3F0E087
:1004F0008081877F8C9380916C008F5F80936C00EC
:1005000080916C00893010F010926C002296F89463
:10051000DEBFCDBFDF91CF91FF91EF91BF91AF9142
:100520009F918F913F912F910F900FBE0F901F9031
:100530001895CF93DF93CDB7DEB780917600909179
:1005400077000097B1F4E6E4F0E080819181909328
:100550007D0080937C00AEE4B0E0EEE4F0E08081CA
:100560008F7B8C9381E090E090937700809376006E
:100570002BC0E6E4F0E08081918190937B00809332
:100580007A00AEE4B0E0EEE4F0E0808180648C9329
:1005900020917A0030917B0080917C0090917D00C9
:1005A000A901481B590BCA019093790080937800E8
:1005B00010927700109276008091780090917900E7
:1005C0009093BF008093BE00DF91CF910895CF93A9
:1005D000DF93CDB7DEB7DF91CF910895CF93DF934F
:1005E000CDB7DEB7E7E2F0E01082E6E2F0E08FEEB2
:1005F0008083DF91CF9108951F920F920FB60F92D3
:1006000011242F933F938F939F93EF93FF93CF9357
:10061000DF93CDB7DEB7E6E2F0E0108280916D00A7
:100620009927E4E2F0E020813181880F991FFC01D5
:10063000EC57FF4F3183208380916D008F5F809353
:100640006D0080916D00883010F010926D00E7E22F
:10065000F0E080916D008083E6E2F0E08FEE808331
:10066000DF91CF91FF91EF919F918F913F912F91CA
:100670000F900FBE0F901F901895CF93DF93CDB7BB
:10068000DEB7E9E2F0E080E18083E0E4F0E01082B0
:10069000EAE2F0E088E18083E0E4F0E086E880834D
:1006A000EBE2F0E082EC8083DF91CF910895CF936D
:1006B000DF93CDB7DEB721970FB6F894DEBF0FBE3C
:1006C000CDBF8983EBE2F0E0808199278072907042
:1006D0000097C1F3ECE2F0E08981808321960FB6A8
:1006E000F894DEBF0FBECDBFDF91CF910895CF93B9
:1006F000DF93CDB7DEB726970FB6F894DEBF0FBEF7
:10070000CDBF9E838D838D819E81DC01FD01019093
:100710000020E9F73197CF018A1B9B0B9C838B83C9
:100720001A8219820FC029813A818D819E81F90137
:10073000E80FF91F80810E94570389819A810196F1
:100740009A83898329813A818B819C8182179307BF
:1007500050F726960FB6F894DEBF0FBECDBFDF91DF
:10076000CF910895CF93DF93CDB7DEB78091690025
:100770000E94570380916A000E945703DF91CF9136
:100780000895CF93DF93CDB7DEB766970FB6F89491
:10079000DEBF0FBECDBF9E8B8D8B8D899E894AE0BB
:1007A00050E09E012F5F3F4FB9010E942504CE010A
:1007B00001960E94770366960FB6F894DEBF0FBECF
:1007C000CDBFDF91CF910895CF93DF93CDB7DEB743
:1007D00022970FB6F894DEBF0FBECDBF8A8387E0A5
:1007E00089831FC08A81482F55278981282F332765
:1007F00027FD309581E090E0022E02C0880F991FFE
:100800000A94E2F7842395231816190624F481E349
:100810000E94570303C080E30E94570389818150DF
:10082000898389818823F4F6809169000E945703A7
:1008300080916A000E94570322960FB6F894DEBF9B
:100840000FBECDBFDF91CF910895FB019F01E894CA
:100850004230C4F04532B4F44A3029F497FB1EF418
:10086000909581959F4F642F77270E945604805D55
:100870008A330CF0895D8193CB010097A1F716F4C0
:100880005DE251931082C9010C944604DC01FC0125
:1008900001900020E9F73297AE17BF0730F47C9142
:1008A0006081708331976D93F7CF0895AA1BBB1BAE
:1008B00051E107C0AA1FBB1FA617B70710F0A61B60
:1008C000B70B881F991F5A95A9F780959095BC0181
:0408D000CD010895B9
:0C08D4004B2000000000003D000D0A0059
:00000001FF
